:1018000050C084C069C068C067C066C065C064C09D
:1018100063C062C061C060C05FC05EC05DC05CC0CC
:101820005BC05AC059C00403090412036F00620070
:101830006400650076002E0061007400100348000B
:101840004900440042006F006F0074001201100153
:1018500000000008C016DF050001010200010902B6
:101860002200010100803209040000010300000091
:10187000092101010001222100070581030800C898
:101880000600FF0901A101150026FF00750885016A
:1018900095060900B20201850295830900B2020192
:1018A000C00011241FBECFE5D4E0DEBFCDBF10E0E5
:1018B000A0E6B0E0E8EBFEE102C005900D92AA368A
:1018C000B107D9F710E0AAE6B0E001C01D92AB392C
:1018D000B107E1F74CD1EEC293CFA82FB92F80E02A
:1018E00090E041E050EA609530E009C02D918227F8
:1018F0009795879510F084279527305EC8F36F5F22
:10190000A8F30895EADF8D939D930895CF93CFB701
:10191000CF93C395B09BE9F7B09B09C0B09B07C0BC
:10192000B09B05C0B09B03C0B09B01C0A3C0DF93B8
:10193000C0917E00DD27CB57DF4FB09B02C0DF9107
:10194000EBCF2F930F931F9306B32FEF00FB20F9DC
:101950004F933F9316B34FEF012700FB21F93BE074
:1019600031C04E7F012F16B3216028C0102F4D7F4C
:101970002260000006B329C04B7F2460012F0000C5
:1019800016B32BC016B3477F28602AC04F7E06B31C
:1019900020612CC04F7D16B320622FC04F7B06B351
:1019A000206432C0422706B349934FEF000010274E
:1019B00010FB20F916B31370C9F1297F91F20127AA
:1019C00000FB21F906B3237F89F2315058F110272B
:1019D00010FB22F916B3277E79F2012700FB23F9C9
:1019E0002F7C81F206B3102710FB24F92F7971F2B6
:1019F00000C016B3012700FB25F92F7359F200C070
:101A000006B3102710FB26F9223040F200C016B3AF
:101A1000012700FB27F9243028F64F77206816B3FA
:101A20000000F9CF10E41ABF002719C03B503195D0
:101A3000C31BD04010E41ABF0881033CF9F00B34FB
:101A4000E9F020917C001981110F1213EDCF4A812A
:101A5000441F093641F10D3211F0013E29F7009380
:101A600083003F914F911F910F912F91DF91CAB742
:101A7000C6FD4FCFCF91CFBFCF9118952091830056
:101A8000222379F310918100112321F5343022F1C2
:101A90003093810020937D0010917E003BE0311B4C
:101AA00030937E0019C00091810001309CF40AE55A
:101AB0004F7081F43091600034FD10C000936000DD
:101AC000C1E7D0E00FC02795A8F45150A9F4220F28
:101AD0000000F9CF4AE503C042ED01C0432FC4E145
:101AE000D0E032E017B31360C09A17BB08B320E40C
:101AF00013E05F93012756E008BB279520F451506F
:101B000021F4220FF9CF012756E000003B5A08BB11
:101B1000D0F2279528F4515029F4220F0000F9CF74
:101B2000012756E0279508BB20F4515021F4220FDD
:101B3000F9CF012756E02991332308BB21F60C7F0A
:101B400010918200110FC651D04008BB11F01093C4
:101B50007C0010E41ABF016017B31C7F402F4C7F3C
:101B60005F9100C000C008BB17BB48BB7ACF84E0C0
:101B700085BB88E28A95F1F79A998BC181E08BBF8A
:101B800082E08BBF85B7836085BF8BB780648BBFD6
:101B9000B89A20E0A89588EB9BE00197F1F72150D7
:101BA000C9F7B8987894FF2400E0A8959091810037
:101BB000392F335037FD19C180917E00ACE0B0E081
:101BC000A81BB109AB57BF4F80917D008D3209F042
:101BD000BDC0383009F007C183EC809371008AE5FD
:101BE0008093600010926A002C91822F807611966B
:101BF0009C9111978823E1F0993079F412968C9199
:101C00001297823031F410926D0027FD8CC09FEF47
:101C10008CC081E080936E004BC1913009F048C1C7
:101C200082E690E09093800080937F0027E081C05F
:101C300012968C91129710927A00992331F4109297
:101C40007B008AE790E022E069C0953019F4809328
:101C5000820061C0963009F04EC013968C911397A4
:101C6000813019F48CE498E11DC0823041F48EE596
:101C700098E19093800080937F0022E238C0833007
:101C800009F512968C911297882341F486E298E127
:101C90009093800080937F0024E029C0813041F43C
:101CA0008AE298E19093800080937F0022E11FC038
:101CB0008230E1F48CE398E19093800080937F0080
:101CC00020E115C0813241F480E798E190938000D3
:101CD00080937F0029E00BC0823241F480E898E1D4
:101CE0009093800080937F0021E201C020E080E497
:101CF00080936A001EC0983019F484E890E009C00F
:101D0000993019F48093840006C09A3021F48AE750
:101D100090E021E003C08AE790E020E0909380000B
:101D200080937F0006C016969C9180E880936A009D
:101D30000AC017968C911797882321F416969C91C8
:101D4000921708F0922F909361004DC080916A0025
:101D500087FF49C0C0916B00D0916C0080916D00ED
:101D6000882349F41196CC9111971296DC91129721
:101D70001496392F3750632F680F60936D00AE01B2
:101D80004F7351F4F89483E0FE0180935700E89577
:101D9000789407B600FCFDCFF894AE018D919C912C
:101DA000119721E0FE010C0120935700E8951124C2
:101DB00078942296FE01EF7351F4F89485E0FA01CD
:101DC00080935700E895789407B600FCFDCF325019
:101DD00011F01296D4CFD0936C00C0936B0067FFC4
:101DE00002C010926100109281008091600084FF17
:101DF0003CC0809161008F3FC1F1182F893008F0FD
:101E000018E0811B809361008091710098E8892718
:101E1000809371001123E1F0E0917F00F091800048
:101E200080916A0086FF09C0912FA2E7B0E08491FB
:101E30008D9331969150D9F707C0912FA2E7B0E06A
:101E400081918D939150E1F7F0938000E0937F00B2
:101E500082E790E0612F56DD612F6C5F6C3019F0E6
:101E60008FEF809361006093600094E186B383708C
:101E700031F49150D9F71092820010927C00809139
:101E80006E00882321F0FA9411F4015011F09A9B0E
:101E90008CCEF89481E180935700E8951BBE15BE67
:101EA00081E08BBF1BBEE0916F00F091700009953F
:081EB00020E03FCFF894FFCFC2
:0A1EB8005AFF014000002000000066
:0400000300001800E1
:00000001FF
